:020000040000FA
:1000000083168E100E141528A6000308A8000408F5
:10001000A7000A08A900622029088A00270884008E
:1000200028088300A60E260E0900FF239000113039
:100030009F008312093085000730990000309F002F
:10004000831609308500D7308100960183128B0119
:10005000203084008001840A2A300402031D2A28EB
:10006000F0308100A0308B000000093085000000D6
:1000700085193528512085193528512085193528AD
:100080005120851935280508363903194B282108D0
:100090002502031C4E28A401A501A00A57208500B3
:1000A00038280330A300A308031D532808002008A4
:1000B000073982070B340D34193429340B340D34CD
:1000C000193429340B1D0800F03081000B11A303F3
:1000D000A40F6B28A50A050836390319080001305A
:1000E0009F007F209F149F1873281E08A1000310F3
:1000F000A10C0310A10CA10A00309F0008000530DC
:08010000A200A20B81280800F7
:02400E00843FED
:00000001FF
